:020000040800F2
:10800000A8810020498100082D9A00080F980008D7
:10801000299A00089D9500085DA300080000000053
:10802000000000000000000000000000259C000887
:108030007D96000800000000B59A0008119D000818
:108040006381000863810008638100086381000880
:108050006381000863810008638100086381000870
:108060006381000863810008638100086381000860
:108070006381000863810008638100086381000850
:108080006381000863810008638100086381000840
:1080900051A3000863810008638100086381000820
:1080A0006381000863810008638100086381000820
:1080B000219E000863810008638100086381000835
:1080C0006381000863810008638100086381000800
:1080D00063810008ED9F0008638100086381000848
:1080E00063810008638100086381000863810008E0
:1080F00063810008638100086381000863810008D0
:1081000063810008638100086381000863810008BF
:108110006381000863810008BD9E00086381000838
:10812000638100086381000863810008638100089F
:10813000DFF810D000F0AAFE00480047D9BE0008C2
:10814000AFF30080A881002006488047064800471A
:10815000FEE7FEE7FEE7FEE7FEE7FEE7FEE7FEE7F7
:10816000FEE7FEE7C19D0008318100082DE9F041DE
:108170000024061B254671F1000605DA01240027BC
:10818000D0EB070067EB0101161E73F1000605DA5C
:108190000027D2EB0702012567EB030300F07AFC0E
:1081A00086460E4617469C46AC4204D00025D0EBCE
:1081B000050E65EB010624B10020D2EB000760EB51
:1081C000030C704631463A466346BDE8F081000034
:1081D0000048704784C8000810B50446FFF7F8FF50
:1081E0000068005D00F0010010BD40EA01039B073C
:1081F00003D009E008C9121F08C0042AFAD203E01C
:1082000011F8013B00F8013B521EF9D27047D2B27F
:1082100001E000F8012B491EFBD270470022F6E76F
:1082200010B513460A4604461946FFF7F0FF2046EC
:1082300010BD421C10F8011B0029FBD1801A7047A9
:108240000FB400B58DB010A909900B9000914FF0BC
:10825000FF300A9000200C900548069005480790D2
:108260006A4609A80F9900F06BFC0DB05DF814FB8D
:108270005D8B00087B8B00082DE9FF4F087883B0E9
:108280009946FF2805D0491C2D2804D00024002041
:1082900008E000200BE00124F9E700EB800003EB8D
:1082A0004000491C0B78FF2BF7D104B1404200235A
:1082B0000293147819461D462D2C01D02B2C04D185
:1082C000521C2D2C13D000240294AA461478FF2CA3
:1082D0000FD00A25A3FB057801FB05814FF0000CA8
:1082E00003FB0C11521CE3194AEB0101EEE70124D8
:1082F000EAE7814453EA010002D019F5C87F06DAA3
:1083000003980021C0E9001107B0BDE8F08F0025F7
:10831000AE4E2F46DFF8B882184600F07AFDCDE960
:108320000001B9F1000002DAC9F1000400E00446DE
:108330000023A74A1AEB030B42EB045A12E0E007B2
:1083400007D02A4633463846414600F00DFA074624
:1083500088462A4633461046194600F005FA054677
:108360000E466410002CEAD1DDE90001B9F1000FDE
:108370005A46534606DA00F069FA3A46434600F098
:1083800065FA05E000F0F0F93A46434600F0ECF9F2
:10839000029A0AB181F00041039AC2E90001B3E7F1
:1083A0002DE9FF4F1F468DB0D7E901464FF0FF384A
:1083B0002E2045464FF000090B90B9696D1C0E98B0
:1083C0008847396A824688470028F6D1BAF1FF3FCC
:1083D0000AD024F4D064002E11DDBAF12B0F08D09E
:1083E000BAF12D0F0BD102E0404611B08DE744F4F5
:1083F0008064B9696D1C0E9888478246761E69466E
:10840000600501D52D2000E02B208DF8000001F142
:10841000010B0DF1200809E0B9696D1C0E98884721
:1084200082460F9844F40074761E0560002E02DD2B
:10843000BAF1300FF0D00B998A453ED144F0800458
:1084400006E00F99681CA9F1010944F40074086062
:10845000B9696D1C761E0E98884782463028F0D088
:108460002BE00B998A4505D1200603D444F0800403
:10847000761E18E0504602F06FF808B30DF11301B4
:10848000761E44F400748B4508D2AAF130000BF834
:10849000010B200607D5A9F1010003E0200602D454
:1084A00009F101008146A00502D50F99681C0860FA
:1084B000B9696D1C0E9888478246002ED1DC53E0C6
:1084C000002E51DDBAF1650F02D0BAF1450F4BD144
:1084D000A00549D5B9696D1C24F44074761E0E9828
:1084E00088478246002E0CDD2B2804D0BAF12D0FD0
:1084F00007D144F48074B9696D1C0E988847824690
:10850000761EE00501D52D2100E02B2108F8011B86
:10851000CDF82C8021E00DF12901761E44F4007481
:1085200088450CD2AAF1300010F0FF0088F8000056
:1085300002D10B99884509D908F1010806E0E00548
:1085400001D5244801E042F20F708146B9696D1CE3
:108550000E98884782460F980560002E04DD50462D
:1085600001F0FAFF0028D6D1F9690E988847FF205C
:108570008BF8000088F800000020069007904B461A
:108580006A4608A906A8FFF777FEA00502D46FF097
:1085900001002AE714F0240F0AD0E00714D1DDE926
:1085A00006123868031D3B600068C0E900120BE04A
:1085B000DDE9060100F028FA0146E00704D1386839
:1085C000021D3A600068016028460EE70000144072
:1085D0000000F03FF1D8FFFFF0B480EA0102D40FB1
:1085E0004200B2EB410F02D20246084611464A0051
:1085F00042D0C30DDDB2C1F3C752AD1A202D35DA1A
:10860000C1F3160141F4000204B15242C5F1200643
:1086100002FA06F12A411044B3EBD05F23D0C4B173
:10862000012DA0EBC35009DCF0BC4FF0004202EA80
:10863000C352DBB200F5000000F0B9BA400000F10F
:10864000807000EBC350A0F1807040EAD170490007
:1086500009E0490841EAC071A0EBC35000F50000F1
:10866000400800EBC350F0BC00F098BA6142012210
:1086700002EB4101001BF6E7F0BC704781F00041BE
:10868000AAE780F00040A7E780EA010210B502F0F7
:108690000043400022D04A001FD0010E01EB1261BE
:1086A000C0F35600C2F3560240F4000042F4000248
:1086B000A0FB022000047F39140400D0401C50EAC3
:1086C000124001D44000491EC2B20C0604EBD01087
:1086D000401C4008802A02D003E0002010BD20F09A
:1086E0000100002900DA0020184310BD30B480EAF0
:1086F000010202F0004530F0004221F0004013D0AA
:1087000090B1C30DD40DC2F31601C0F31600E41AE4
:1087100041F4000140F400027D34914201D3641C15
:1087200000E04900002C02DA30BC002070474FF412
:1087300000000023914201D3891A034340084FEA05
:108740004101F7D151B1914202D14FF0004105E012
:1087500002D24FF0010101E06FF0010103EBC450C0
:10876000284430BC00F01ABA2DE9FE4F81EA030418
:1087700004F0004421F0004100944FF0000B23F07E
:10878000004350EA01045ED052EA03045BD0C3F315
:108790000A54C1F30A552C44A4F2F3340194A0FB0B
:1087A0000254C1F3130141F48011C3F3130343F4E2
:1087B000801301FB024400FB034E840A970A44EA3B
:1087C000815447EA8357A4FB076802958D0A05FB8D
:1087D00007854FEA932C04FB0C542705029D4FEAB2
:1087E000065847EA1637B5EB08056EEB070C870EFF
:1087F000920E47EA811742EA8312A7FB0201B6EB09
:108800000B0164EB00042B0D43EA0C335E1844EBC0
:108810001C50DA465146E7FB0201C5F313044FEA48
:108820000B3343EA14534FEA0432019C43EA060334
:10883000A4F10C040294009CCDE900B400F0F4F91A
:1088400003B0BDE8F08F00200146F9E72DE9F04DB7
:1088500081EA030404F0004B21F0004514464FF078
:10886000000A23F0004150EA050220D054EA010238
:108870001DD0C5F30A570246C5F31303C1F3130015
:10888000C1F30A5640F4801543F48013A7EB0608A1
:10889000101BD64608F2FD3873EB050002D308F131
:1088A000010801E092185B41B8F1000F03DA0020E3
:1088B0000146BDE8F08D00204FF480110646844645
:1088C0000EE0171B73EB050705D3121B63EB0503C3
:1088D00006434CEA010C49084FEA300092185B410C
:1088E00050EA0107EDD152EA030012D082EA0400F7
:1088F00083EA0501084305D0101BAB4106D20122D3
:10890000002306E000224FF0004302E06FF0010276
:1089100053101AEB06004CEB085110EB0A0041EB28
:108920000B01BDE8F04D00F070B9C10F80EAE070B6
:108930000844CA079623002100F039B99623002283
:10894000114600F034B900F0004220F00040C10DA3
:10895000C0F3160040F400007F2901DA00207047C0
:10896000962903DCC1F19601C84001E096398840A0
:10897000002AF4D04042704720F00040C10DC0F3FF
:10898000160040F400007F2901DA00207047962984
:1089900003DCC1F19601C8407047963988407047A2
:1089A00010B500F0004420F00040C20DC0F31600E6
:1089B00040F400007F2A02DA0020014610BD0021A9
:1089C000962A03DCC2F19602D04002E0963A00F00B
:1089D00092F8002CF2D00023D0EB030063EB0101EE
:1089E00010BD00F0004230F000400AD0C10D01F58A
:1089F0006071C0F3160042EA0151C20840071143FA
:108A0000704700200146704701F0004330B421F068
:108A1000004150EA010206D00A0DA2F56072C1F3CE
:108A20001301002A02DC30BC00207047440F44EAE6
:108A3000C104C100E01830BC00EBC25000F0AEB879
:108A4000002801DBC0F10040002901DBC1F1004139
:108A500081427047002801DBC0F10040002901DBA2
:108A6000C1F100418842704730B50B4601460020F5
:108A70002022012409E021FA02F59D4205D303FAE0
:108A800002F5491B04FA02F52844151EA2F1010261
:108A9000F1DC30BD2DE9F05F0546002092469B4693
:108AA00088460646814640241BE028464146474604
:108AB000224600F02FF853465A46C01A914110D36F
:108AC00011461846224600F016F82D1A67EB0108E9
:108AD0004F4622460120002100F00DF817EB000957
:108AE0004E41201EA4F10104DFDC484631462A46EF
:108AF0004346BDE8F09F202A04DB203A00FA02F149
:108B0000002070479140C2F1200320FA03F319437B
:108B100090407047202A04DB203A21FA02F000211D
:108B2000704721FA02F3D040C2F12002914008437D
:108B3000194670470268114413780160184670475F
:108B4000D16004495161044911620021116111464B
:108B500000F0C0B9358B0008D9810008426842B1E5
:108B6000016811F8013B23B1521EC0E900121846FA
:108B700070470121C160881E704742685AB1C368BE
:108B8000016843B983688B4205D0491E521CC0E975
:108B90000012002070474FF0FF3070470029A8BF37
:108BA0007047401C490008BF20F00100704710B416
:108BB000B0FA80FC00FA0CF050EA010404BF10BCCB
:108BC000704749B1CCF1200421FA04F411FA0CF1F8
:108BD00018BF012121430843A3EB0C01CB1D4FEA31
:108BE00000614FEA102042BF002010BC704700EB2C
:108BF000C35010440029A4BF10BC7047401C49005A
:108C000008BF20F0010010BC704710B5141E73F1AE
:108C1000000408DA401C41F1000192185B411A433C
:108C200001D120F0010010BD2DE9F04D92469B4688
:108C300011B1B1FA81F202E0B0FA80F2203290462E
:108C4000FFF759FF04460F4640EA0A0041EA0B01CC
:108C500053465A46084313D0114653EA010019D02F
:108C6000C8F140025046FFF755FF05460E465046F4
:108C700059464246FFF73FFF084305D0012004E074
:108C800020463946BDE8F08D0020054346EAE076EF
:108C90002C4337430A986305E40AA0EB080000223E
:108CA000FD0A44EA47540A3002D500200146E9E7AC
:108CB000010510196941DDE9084500196941BDE860
:108CC000F04DA2E72DE9FE4F804681EA0300C00F78
:108CD0000C46009021F0004123F00045B8EB020063
:108CE000A94105D24046214690461C460B46024605
:108CF00023F00040104347D0270DC7F30A00C3F309
:108D00000A510290401A019040286BDAC3F3130015
:108D100040F4801B0098924620B10023D2EB030A56
:108D200063EB0B0B01985946C0F140025046FFF728
:108D3000E2FE06460D4650465946019A00F0B8F844
:108D400010EB08006141002487EA115284EAE773BE
:108D50001A4340D0009A62B3019A012A4FEA07529F
:108D600015DC001B61EB02014FF0004202EA0752E2
:108D7000CDE90042001C41F5801132462B46FFF739
:108D800053FF03B0BDE8F08F40462146F9E7001BD2
:108D900061EB0201001C41F5801300185B412018B3
:108DA000A2F5001747EB030140EAD570B6196D41F3
:108DB00011E06D084FEA360645EAC0754FEA0752E2
:108DC000001B61EB0201001C41F5801149084FEACC
:108DD00030000019514132462B4603B0BDE8F04F38
:108DE000FFF713BF0098012240000023D0EB0202DE
:108DF00063EBE073009821464FEAE074B8EB0000A3
:108E000061EB0401E9E783F000435BE781F0004197
:108E100058E70EB540F2334202920022CDE900221B
:108E20001346FFF701FF03B000BDC1F30A52C1F3BF
:108E3000130140F2FF3341F480119A4202DA00201C
:108E40000146704740F233439A42A2F2334202DCB9
:108E50005242FFF75FBEFFF74EBE000030B5041E62
:108E600071F1000404DB4FF00044404264EB010167
:108E7000141E73F1000405DB1C464FF00043524200
:108E800063EB0403994208BF904230BD064C074D86
:108E900006E0E06840F0010394E8070098471034CA
:108EA000AC42F6D3FFF748F92CC900084CC90008BA
:108EB000202A06DBCB17203A41FA02F043EAE0739E
:108EC00006E041FA02F3D040C2F12002914008438B
:108ED000194670472DE9F34F8BB04FF0000801F1B0
:108EE0000C000C464FF0010B46460DF1080A0190AC
:108EF0006269012101989047051E2DD0252D2CD0A7
:108F0000216A8847C0B16269012101989047216AAE
:108F100088470028F7D1411E62690198904700E018
:108F2000761CA1690B988847216A88470028F7D1E9
:108F3000E1690B988847DBE7A1690B9888470746EA
:108F4000A84201D1761CD3E7E1690B9888477F1CC2
:108F500002D1B8F1000F6FD047E1002762693D46AA
:108F60003946019890472A2804D162690121019865
:108F700090470125DFF888926269012101989047A6
:108F8000A0F130010A290AD24F45E5DC07EB870141
:108F900000EB4107303FDFD445F01005ECE7E90670
:108FA00001D46FF000476C280AD04C2814D06828F0
:108FB00015D06A280DD074281CD07A281AD01DE04C
:108FC00062690121019890476C2802D045F00405A0
:108FD00014E045F002050DE045F020050AE0626965
:108FE000012101989047682802D045F0080505E066
:108FF00045F400656269012101989047C4E9015771
:1090000065283DD019DC58287AD00CDC452837D0AB
:1090100004DC252826D0412831D131E046282FD044
:1090200047282CD12CE05B2877D0612828D06328F2
:109030007CD0642823D15AE0D1E06F2848D008DCE6
:1090400066281DD067281BD0692821D06E2816D12C
:1090500027E0702845D0732868D0752847D0782835
:109060000DD14DE0A1690B988847054625283FF4AE
:1090700069AFE1690B9888476D1C3FF46AAFB4E0B3
:1090800023466A466FF001000B99FFF789F99FE0CC
:1090900045F040006060A80723464FF0000236D438
:1090A0003EE0E8077FF447AF2068011D21600068BB
:1090B000290501D506701BE7290701D5068017E7AA
:1090C000A90703D5F117C0E9006111E706600FE7B2
:1090D00045F040006060A80723464FF0080216D410
:1090E0001EE040F60E0125EA0100606016E045F042
:1090F00040006060A80723464FF00A0207D40FE043
:1091000045F040006060A80708D5234610226FF0A4
:1091100001000B99AFF300805AE007E023461022CC
:109120006FF001000B99AFF3008051E04FF00009A0
:109130004F464B46632802D05B2807D041E0207998
:10914000C00601D40120A06001273AE06269012134
:10915000019890475E2805D14FF0010962694946A0
:1091600001989047216939B900210A46534643F8CE
:109170002120491C0829FADBB0B3216969B9C1175C
:1091800000EBD16253110AEB830122F01F02821A15
:1091900001200B68904003430B6062690121019834
:1091A00090475D28E8D1B9F1000F09D00020514661
:1091B00051F82020D24341F82020401C0828F7DB3A
:1091C00002AB224600976FF001000B99AFF30080CD
:1091D00000280CDA401C08D1BBF1000F05D04FF07D
:1091E000FF300DB0BDE8F08FFFE74046F9E7E90733
:1091F00001D108F1010806444FF0000B78E60000A9
:10920000CCCCCC0C21B1826842F00102826003E038
:10921000826822F0010282607047000010B50446A7
:109220001248844208D10121401500F081FC002140
:10923000601500F07DFC17E00D48844208D1012143
:10924000001500F075FC0021201500F071FC0BE00A
:109250000848844208D10121C80300F069FC0021BC
:109260004FF4004000F064FC10BD000000240140F9
:1092700000280140003C0140014600208A6802F0BD
:1092800004020AB1012000E0002070470146C86CCA
:1092900080B270470246002013680B400BB10120DA
:1092A00000E000207047014600208A6802F00802B2
:1092B0000AB1012000E000207047000030B50246EE
:1092C0000020002350680F4C20400D790C6844EAC0
:1092D00005242043506090680B4C2040D1E9025493
:1092E0002C434D7944EA450420439060D06A20F431
:1092F00070000C7C641EE4B2234340EA0350D06249
:1093000030BD0000FFFEF0FFFDF7F1FFF0B50446B1
:109310000D4600200021092D11DDE068A5F10A06A7
:1093200006EB4607072606FA07F18843A5F10A0669
:1093300006EB460603FA06F10843E0600CE02069FC
:1093400005EB4507072606FA07F1884305EB4506B6
:1093500003FA06F108432061072A0FDA606B561EF4
:1093600006EB86071F2606FA07F18843561E06EB12
:10937000860605FA06F10843606322E00D2A0FDA3B
:10938000206BD61F06EB86071F2606FA07F18843D7
:10939000D61F06EB860605FA06F10843206310E0A7
:1093A000E06AA2F10D0606EB86071F2606FA07F112
:1093B0008843A2F10D0606EB860605FA06F108437E
:1093C000E062F0BD816841F008018160704721B121
:1093D000826842F4A002826003E0826822F4A00264
:1093E00082607047816841F004018160704700002D
:1093F00000B587B001214FF4017000F089FB4FF4F4
:10940000004000F059FB0620ADF8040000208DF864
:10941000070001A9174800F03CF91748FFF7FEFEC6
:10942000002002908DF80C008DF80D004FF46020A4
:1094300004900020059001208DF8180002A90E4824
:10944000FFF73CFF01210C48FFF7DCFE0A48FFF75D
:10945000B9FF00BF0848FFF726FF0028FAD10648E9
:10946000FFF7C0FF00BF0448FFF706FF0028FAD14E
:1094700007B000BD000801400024014008B50121EB
:10948000082000F045FB4FF4807008490860032075
:109490008DF8020010208DF803000001ADF80000E7
:1094A00069460248143800F0F4F808BD140C014075
:1094B00000B501231A46042141F2CC0000F056F811
:1094C00000BD00002748007810B12648808800B908
:1094D000704724484078B0B92248808800283FDD92
:1094E00020480089401C80B21E4908814988884272
:1094F00036DB4FF480701C49086000201949088150
:10950000012048702CE017484078012828D11548E0
:109510000089401C80B213490881898888421FDB7A
:109520001048C088002812DD0E484089401C80B2D7
:109530000C494881C988884202DB0020094908702B
:109540000848007818B9002006498880C0E7002044
:109550000449088148704FF480700349091F08606E
:1095600000BFB5E770000020140C014030B501B910
:1095700030BD084CE0606180A280E3800024054D8E
:109580002C816C816C7001242C702402024D2C60A3
:1095900000BFEDE770000020100C014000BFFEE7A7
:1095A00039B1084A1268012383401A43054B1A60F7
:1095B00006E0044A1268012383409A43014B1A6073
:1095C000704700000074004030B5002200230A4CB0
:1095D000226840F6FE748440A243D1E900452C4342
:1095E0008D682C43CD6844EA050303FA00F4224356
:1095F000014C226030BD00000074004008B500221C
:109600000092054A009200F10802009B1A44009261
:10961000009A116008BD00000074004021B102688A
:1096200042F00102026004E002684FF6FE731A4045
:10963000026070470146486880B2704710B500224A
:10964000026847F6F0739A430C6A8B6823430C69EF
:1096500023434C6923438C692343CC6923434C6ADD
:1096600023438C6A23431A430260CB6843600B6830
:1096700083604B68C36010BD416070477047002134
:1096800001E04A1C91B24FF4967242438A42F8DCE0
:1096900070472DE9F04102460025002600200023F6
:1096A0000024002791F803C00CF00F0591F803C0C7
:1096B0000CF0100CBCF1000F03D091F802C04CEA82
:1096C000050591F800C0BCF1000F31D014680020EE
:1096D0002BE04FF0010C0CFA00F3B1F800C00CEADB
:1096E00003069E4220D183004FF00F0C0CFA03F7C3
:1096F000BC4305FA03FC4CEA040491F803C0BCF136
:10970000280F06D14FF0010C0CFA00FCC2F814C06F
:109710000AE091F803C0BCF1480F05D14FF0010CED
:109720000CFA00FCC2F810C0401C0828D1D3146009
:10973000B1F800C0BCF1FF0F34DD546800202EE00A
:1097400000F1080C4FF0010808FA0CF3B1F800C062
:109750000CEA03069E4221D183004FF00F0C0CFA55
:1097600003F7BC4305FA03FC4CEA040491F803C078
:10977000BCF1280F05D100F1080C08FA0CF8C2F86A
:10978000148091F803C0BCF1480F07D100F1080C18
:109790004FF0010808FA0CF8C2F81080401C0828A5
:1097A000CED35460BDE8F0810161704710B5044626
:1097B0000723012221460948FFF7A8FD0121074898
:1097C000FFF705FE00BF02210448FFF763FD0028F4
:1097D000F9D00248FFF75AFD10BD000000240140F7
:1097E0002DE9F04107460C460025002608E03846E2
:1097F000FFF7DCFF05440520FFF741FF701CC6B2F0
:10980000A642F4DBB5FBF4F080B2BDE8F08100BF06
:10981000FEE700000448006800F0080008B90120D5
:1098200070470020FCE70000080801400448006879
:1098300000F0040008B9012070470020FCE7000098
:10984000081801400448006800F0080008B9012029
:1098500070470020FCE70000081801402DE9F041A6
:109860003C48007E08B9BDE8F0813A48407E10B11E
:1098700001286BD14EE001203649487680203649D8
:1098800008613448D0E90810324AC2E90C10104689
:10989000D0E90830D2E90A12591A904109DA2D4864
:1098A000D0E90810491C40F100002A4AC2E908101A
:1098B00011E02848D0E90A202649D1E90831D21A16
:1098C000884108DA2348D0E90810491E60F10000F9
:1098D000204AC2E908101F4842F20D120023D0E9C5
:1098E0000C412046FEF742FC06460F46194842F25C
:1098F0000D120023D0E908412046FEF737FC464010
:109900004F403E4305D01548006880F040001349A1
:1099100008601CE000200F49487680200E4948610D
:109920000C480069401C0B4908610846D0E9081042
:10993000084AD2E90A3259405040014305D100F0AB
:109940003BF80121064800F0D5FA00E000BF00BF57
:1099500000BF88E7C0000020001001400C08014053
:109960000010004070B504460D461646012002F076
:10997000AFF80F48057044608660C66000200C494F
:109980000861012008762DB1012D07D1002002F0D9
:1099900083F804E0012002F07FF800E000BF00BF80
:1099A000610000231A46034801F0DCFD70BD000091
:1099B000C00000200010004010B500231A461946D0
:1099C000084801F0CFFD00200749087680200749AC
:1099D00048610748C07A022802D100200449C872B1
:1099E00010BD000000100040C00000200010014029
:1099F0005400002010B5FFF7DFFF0021084A9162F4
:109A0000D1621162516211635163402005490860BF
:109A100003230522114640F2DC50FFF7A7FD10BDDD
:109A2000C00000201408014000BFFEE7704700009E
:109A300070B5002100230F22C47804B3154C2468AC
:109A400004F4E064C4F5E064210AC1F10403CA40EF
:109A5000447804FA03F184781440214309010E4C40
:109A60000678A155047804F01F050124AC40057860
:109A70006D11AD0005F1E025C5F8004109E004785D
:109A800004F01F050124AC40044D0678761145F81A
:109A9000264070BD0CED00E000E400E080E100E055
:109AA00002490143024A1160704700000000FA05B4
:109AB0000CED00E07047000001460020034A5068AA
:109AC00020F44040084350607047000000100240FE
:109AD00029B1064A52690243044B5A6104E0034A21
:109AE00052698243014B5A617047000000100240E6
:109AF00029B1064AD2690243044BDA6104E0034A01
:109B0000D2698243014BDA617047000000100240C5
:109B100029B1064A92690243044B9A6104E0034A60
:109B200092698243014B9A61704700000010024025
:109B300029B1064AD2680243044BDA6004E0034AC2
:109B4000D2688243014BDA60704700000010024087
:109B500030B500210022002400232D4D6D6805F052
:109B60000C0121B1042905D0082923D105E0294D94
:109B7000056022E0274D05601FE0254D6D6805F466
:109B80007012234D6D6805F48034022505EB924276
:109B90001CB9214D554305600BE01D4D6D6805F462
:109BA00000351DB11C4D5543056002E0194D55436C
:109BB000056002E0174D056000BF00BF144D6D68E1
:109BC00005F0F0010909154D6B5C0568DD40456045
:109BD0000F4D6D6805F4E061090A104D6B5C456836
:109BE000DD4085600A4D6D6805F46051C90A0B4D72
:109BF0006B5C4568DD40C560054D6D6805F440410E
:109C0000890B074D6B5CC568B5FBF3F5056130BD8D
:109C10000010024000127A0000093D0026000020DA
:109C200036000020704710B500F002F810BD0000AB
:109C30000CB50020019000903348006840F480305B
:109C40003149086000BF3048006800F400300090DF
:109C50000198401C0190009818B90198B0F5A06FC8
:109C6000F1D12948006800F4003010B101200090C3
:109C700001E0002000900098012843D123480068AB
:109C800040F01000214908600846006820F00300F9
:109C900008600846006840F0020008601A48406802
:109CA000194948600846406848600846406840F4E2
:109CB000806048600846406820F47C104860084690
:109CC000406840F4E81048600846006840F0807042
:109CD000086000BF0C48006800F000700028F9D050
:109CE0000948406820F0030007494860084640687A
:109CF00040F00200486000BF0348406800F00C00DC
:109D00000828F9D10CBD00000010024000200240DC
:109D100010B500F001F810BD10B52248006840B140
:109D200020480068401E1F49086010B901201E49E4
:109D30000870002408E004EB44011C4A02EB810097
:109D400001F016FD601CC4B2042CF4DB1848006856
:109D5000401C1749086017480088401C15490880B6
:109D600008460088642804DD00200880012012498C
:109D700008700F4800686FF00041884202D100204F
:109D80000B49086001F0EAFB0C480078401CC0B2A7
:109D90000A4908700A2803DB0020087001F0D8FB8C
:109DA00010BD00000400002008000020F800002082
:109DB0000C000020100000200000002024000020E3
:109DC00010B51348006840F00100114908600846CA
:109DD0004068104908400E494860084600680E492E
:109DE00008400B4908600846006820F4802008609D
:109DF0000846406820F4FE0048604FF41F00886069
:109E0000FFF711FF4FF000600449086010BD00002B
:109E1000001002400000FFF8FFFFF6FE08ED00E032
:109E200010B50221480700F074F858B10221480724
:109E300000F060F800220221480700F07BF81B4880
:109E4000006880470421080700F063F858B1042136
:109E5000080700F04FF800220421080700F06AF814
:109E60001348006880470821C80600F052F858B12E
:109E70000821C80600F03EF800220821C80600F0BC
:109E800059F80C48006880471021880600F041F816
:109E900058B11021880600F02DF800221021880604
:109EA00000F048F804480068804710BD1400002006
:109EB000180000201C0000202000002010B5012107
:109EC000054800F026F828B1FFF7C8FC0121024838
:109ED00000F010F810BD00000010004021B1028811
:109EE00042F08002028004E002884FF67F731A403D
:109EF00002807047CA430282704721B1028842F053
:109F00000102028004E002884FF6FE731A400280CC
:109F1000704730B50246002000230024158A05EA68
:109F20000103958905EA010413B10CB1012000E099
:109F3000002030BD1AB183890B43838102E08389FD
:109F40008B43838170470000002202881D4B98429A
:109F50000ED01D4B98420BD0B0F1804F08D01B4B58
:109F6000984205D01A4B984202D01A4B984204D11D
:109F70004FF68F731A404B881A43174B984207D0FD
:109F8000164B984204D04FF6FF431A40CB881A4331
:109F900002808B8883850B8803850A4B98420BD0FF
:109FA000094B984208D00E4B984205D00D4B984271
:109FB00002D00D4B984201D10B7A03860123838294
:109FC00070470000002C01400034014000040040B4
:109FD00000080040000C0040001000400014004049
:109FE00000400140004401400048014010B540F2EB
:109FF0002441174800F0BAF8012827D1002115485C
:10A00000FFF70CFB1348FFF715FB044640211248ED
:10A01000FEF704F9C4F1400210490F48FEF7E5F8D5
:10A0200040210E48FEF7FAF801200D490870402142
:10A030000848FFF721FB01210648FFF7EFFA044823
:10A0400000F050F91021024800F00CF810BD00009B
:10A05000003801405800024068010020280100201B
:10A060002500002001F40072B2F5007F00D100BF8E
:10A07000CA430280704721B1828942F40052828132
:10A0800004E082894DF6FF731A4082817047000018
:10A0900000B587B001210420FFF73AFD01218803B4
:10A0A000FFF736FD4FF4A060FFF7FAFC25208DF88E
:10A0B000040001208DF807008DF8050003208DF8BD
:10A0C000060001A8FFF7B4FC4FF40070ADF81800CB
:10A0D00018208DF81B0003208DF81A0006A91648D9
:10A0E000FFF7D7FA4FF48060ADF8180004208DF820
:10A0F0001B0006A91048FFF7CCFA4FF4E13002909C
:10A100000020ADF80C00ADF80E00ADF81000ADF871
:10A1100014000C20ADF8120002A9084800F076F8EF
:10A12000012240F22441054800F04AF80121034889
:10A13000FFF7A1FF07B000BD000801400038014053
:10A140001AB1838A0B43838202E0838A8B43838222
:10A15000704702460020B1F5007F00D100BF138890
:10A160000B400BB1012000E00020704770B50246A3
:10A17000002400230025002040F66A16B14200D1D9
:10A1800000BFC1F3421501F01F03012606FA03F3D5
:10A19000012D02D19689334006E0022D02D1168AA4
:10A1A000334001E0968A33400C12012606FA04F48B
:10A1B0001688344013B10CB1012000E0002070BDBE
:10A1C000F0B50346002400260025002040F66A175B
:10A1D000B94200D100BF1846C1F3421401F01F0676
:10A1E000012707FA06F5012C01D10C3004E0022CFE
:10A1F00001D1103000E014301AB107682F43076016
:10A2000002E00768AF430760F0BD00002DE9F047AA
:10A2100086B005460E460024A24600BFA146002790
:10A22000B08900B100BF2F462C8A4CF6FF70044065
:10A23000F08804432C82AC894EF6F3100440B088B9
:10A2400031890843718908430443AC81AC8A4FF6D5
:10A25000FF400440B0890443AC8201A8FFF778FCBA
:10A260001F48874202D1DDF810A001E0DDF80CA004
:10A27000A88900F4004040B10AEBCA0000EB0A10C4
:10A2800031684900B0FBF1F807E00AEBCA0000EBC7
:10A290000A1031688900B0FBF1F86420B8FBF0F0D7
:10A2A00004012009642101FB1089A88900F4004001
:10A2B00040B1322000EBC900B0FBF1F000F0070024
:10A2C000044308E0322000EB09106421B0FBF1F0F8
:10A2D00000F00F0004432C8106B0BDE8F0870000B9
:10A2E0000038014001468888C0F308007047C1F378
:10A2F000080282807047000000B58BB0012108463B
:10A30000FFF7E6FB0F4800900F48019000200290F5
:10A3100040200390002004908020059000200690AB
:10A32000079020200890C001099000200A906946FB
:10A330000648FFF783F901210448FFF76FF90BB0D6
:10A3400000BD0000043801402801002058000240F0
:10A350000148C069704700000010024000BFFEE7DE
:10A360000FB4054B10B503A9044A029800F0FCF89D
:10A3700010BC5DF814FB0000E9BC00085000002090
:10A380000FB47CB50C0009AD01D0611E00E00021C6
:10A39000CDE90001064B6A462946089800F0E4F82A
:10A3A000002C02D0009A002111707CBC5DF814FBD7
:10A3B0006FAC000802E008C8121F08C1002AFAD1D9
:10A3C00070477047002001E001C1121F002AFBD135
:10A3D000704700002DE9FF5F82B00021DDE9043005
:10A3E000020DDDF840B0034318D044F61050A2F23D
:10A3F000FF3242431514119801281FD0A5EB0B0022
:10A40000401C5FEA000A4FF000064E4FDFF838911B
:10A41000B046504615D5CAF1000413E01198012446
:10A420004AA3012801D16FEA0B010298119AC0E9F1
:10A430000031C0E9024206B0BDE8F09FCBF1000058
:10A44000DFE704460021404A491842EB0450CDE9B9
:10A45000001012E0E00707D032463B46404649462E
:10A46000FEF782F98046894632463B461046194639
:10A47000FEF77AF906460F466410002CEAD1DDE9B2
:10A480000401DDE90023BAF1000F06DAFEF76CF9EA
:10A4900042464B46FEF768F905E0FEF7D7F942461B
:10A4A0004B46FEF7D3F904460E460022284BFEF732
:10A4B000D5FC03D84FF0FF30014607E00022254BC2
:10A4C00020463146FEF7FEFBFEF7AFFC102409E004
:10A4D000002C0ADB0A220023FEF7DCFA039B303251
:10A4E0001A55641E50EA0102F2D1641C039AC4F1A9
:10A4F00011031444119A012A03D0012208430DD1FB
:10A500000AE0084304D000204FF0110B119072E7CD
:10A51000A3EB0B056D1E0DE05B4504DD4FF0000263
:10A5200005F1010504E003DA4FF00002A5F1010591
:10A53000002AECD002981199C0E90231C0E9004527
:10A5400079E70000000014400000F03F30000000F8
:10A550000000F0430000E03F30380A2801D201201B
:10A5600070470020704700002DE9FF4F95B09A46D4
:10A57000884606460025EEE1252877D100242746A7
:10A58000F94A0121039400E0044316F8013F203BFF
:10A5900001FA03F01042F7D130782A2811D06FF079
:10A5A0002F033078A0F13002092A16D8039A44F01C
:10A5B000020402EB820203EB42021044761C039079
:10A5C000EFE758F8042B0392002A03DA504244F4D0
:10A5D0000054039044F00204761C30782E2816D1E3
:10A5E00016F8010F44F004042A280DD06FF02F0252
:10A5F0003078A0F13003092B09D807EB870302EB71
:10A600004303C718761CF3E758F8047B761C3078B0
:10A610006C280FD006DC4C2817D068280DD06A288B
:10A6200014D104E0742810D07A280FD10DE044F43E
:10A6300000140AE044F4801401E044F440147278F9
:10A64000824202D104F58014761C761C307866288C
:10A650000BD013DC582877D009DC002875D04528AA
:10A66000F6D04628F4D047281AD193E118E06328A1
:10A6700035D0642879D0652812D18BE1702873D049
:10A6800008DC6728F1D069286FD06E280DD06F28BC
:10A6900006D1ACE073282CD0752874D0782853D01C
:10A6A0005246179990476D1C54E1C4F3025002289A
:10A6B00009D003280DD0D8F8001004280DD00D6063
:10A6C00008F1040846E1D8F80010EA17C1E9005281
:10A6D000F6E7D8F800100D80F2E70D70F0E718F8F3
:10A6E000041B8DF8001000208DF80100EB460120BE
:10A6F00003E058F804BB4FF0FF3061074FF0000152
:10A7000002D40DE009F101018946B9420FDA814511
:10A71000F8DB1BF809100029F4D108E009F1010168
:10A7200089468142FADB1BF809100029F6D103980B
:10A730005346A0EB090721463846179A00F080FAE5
:10A74000284400EB090507E044E008E10DE01BF8B0
:10A75000010B524617999047B9F10109F7D25346B8
:10A7600021463846179AF2E039E00A21C4F3025232
:10A770004FF0000B0091022A06D058F8040BC117C5
:10A78000032A09D00AE023E008F1070020F00702BD
:10A79000F2E80201904605E000B2C117042A01D197
:10A7A00040B2C117002906DA0A460021404261EB97
:10A7B00002012D2202E0220504D52B228DF804206F
:10A7C000012203E0E20701D02022F7E7914657E09B
:10A7D0000A2100E010214FF0000B00910BE0102146
:10A7E0004FF0000B44F004040827009103E0082018
:10A7F0004FF0000B0090C4F30252022A05D058F823
:10A80000040B0021032A08D008E008F1070020F01B
:10A810000702F2E80201904603E080B2042A00D168
:10A82000C0B24FF0000922072AD53278702A07D02B
:10A83000DDF800C08CF0100C5CEA0B0C05D00EE0CB
:10A8400040228DF80420012208E050EA010306D0DE
:10A8500030238DF804308DF8052002229146009BAC
:10A8600083F0080353EA0B030AD150EA010201D135
:10A87000620705D530228DF804204FF001097F1EB4
:10A880003278582A04D039A20C920CAA02920BE01A
:10A890003BA2F9E75B46009AFEF7FCF80C9B9B5C39
:10A8A000029A521E0292137050EA0102F2D10298EB
:10A8B00004A9081A00F1200B600702D524F48034A3
:10A8C00000E001275F4502DDA7EB0B0000E0002060
:10A8D00000EB0B01009003984944401A0390E003F9
:10A8E00006D453462146179A039800F0A9F9054467
:10A8F000002706E001A85246C05D179990476D1CDD
:10A900007F1C4F45F6DBE0030CD553462146179AD2
:10A91000039800F095F9054404E030205246179959
:10A9200090476D1C0099481E00900029F5DC08E056
:10A930000298029952460078491C02911799904753
:10A940006D1CBBF10001ABF1010BF1DC5BE100F030
:10A9500065F90544761C307800287FF40DAE19B0F7
:10A960002846BDE8F08F000009280100303132335D
:10A97000343536373839616263646566000000003B
:10A980003031323334353637383941424344454625
:10A9900000000000600700D4062708F1070020F03F
:10A9A0000700F0E80223804603F0004C5FEA0C0049
:10A9B00001D097A009E0200501D596A005E0E007A9
:10A9C00001D095A001E0AFF24C001390307823F055
:10A9D000004365280CD006DC452809D046281DD048
:10A9E00047287FD13BE0662818D067287AD136E027
:10A9F0000021112F01DB112000E0781CCDE90001BE
:10AA000004A90CA8FFF7E6FCDDE90D010C9A4FF054
:10AA1000000B07F10109109200914EE04FF0004049
:10AA20000097CDE9011004A90CA8FFF7D3FCDDE9DC
:10AA30000D020C9B0F994FF0000B91461093009262
:10AA400011B9791C00EB0109B7EB090003D4C0F17F
:10AA5000FF3B07F10109A9EB0700019042E0012F3C
:10AA600000DA01270021112F01DD112000E0384616
:10AA7000CDE9000104A90CA8FFF7ACFCDDE90D014C
:10AA80000C9A00914FF0000BB946109221070FD499
:10AA9000009A4A4503DA914601E0A9F10109B9F1AA
:10AAA000010F05DD109AA9F10101515C3029F4D0A4
:10AAB000B84202DA10F1040F03DA0121CDE90110E6
:10AAC00010E0002803DC8344A9EB000102E0411CF4
:10AAD000494500DD8946A0EB0B00401C01904FF07A
:10AAE00000400290200705D40198484502DB4FF052
:10AAF000FF30019000208DF84B0002980DF14B07BC
:10AB0000B0F1004F25D002200C902B200D90029820
:10AB100000280CDA404202902D200D9007E00A2117
:10AB20000298FDF7A1FF3031029007F8011D0C9942
:10AB3000481E0C900029F2DC02980028EFD1791E03
:10AB40000D980870307800F0200040F0450007F8BC
:10AB5000020D11A8C01BC01D02901398007800B10F
:10AB6000012000EB0901019801EBE071029801441A
:10AB70000398401A401E0390E00306D45346214632
:10AB8000179A039800F05CF805441398007818B100
:10AB90005246179990476D1CE00323D55346214632
:10ABA000179A039800F04CF805441BE0BBF1000F26
:10ABB00007DB0098584504DD1098179910F80B0032
:10ABC00001E0179930205246904701980BF1010B94
:10ABD000401E05F10105019004D12E20524617991F
:10ABE00090476D1CB9F10001A9F10109DEDC05E017
:10ABF00017F8010B5246179990476D1C0299481E91
:10AC000002900029F4DC53462146179A03989EE6E9
:10AC10002D0000002B000000200000002DE9F04175
:10AC2000044600251E461746880404D405E039462C
:10AC30002020B0476D1C641EF9D52846BDE8F08180
:10AC40002DE9F041044600251E469046C80301D573
:10AC5000302700E02027880404D505E04146384627
:10AC6000B0476D1C641EF9D52846BDE8F0814A68DE
:10AC7000002A06D00A68531C0B6010704868401EFA
:10AC8000486070472DE9F04100243848006942F2DD
:10AC90000D1190FBF1F201FB1200084490FBF1F260
:10ACA00001FB12084046FDF740FE07463049FDF71C
:10ACB000EBFC06462F49FDF719FD05460021284605
:10ACC000FDF7BEFE0BD24FF07C512846FDF7D6FCB7
:10ACD000054627492846FDF77FFC054605E04FF06D
:10ACE0007C512846FDF778FC05462048002101608C
:10ACF00041602846FDF727FE1C49886108461EA2D0
:10AD000009218369FFF73CFB00242AE01748005D16
:10AD1000202807D10B2015490855052C1FDB0020E2
:10AD200008551CE01148005D2D280BD1052C05DBD2
:10AD30000A200E4908710020085510E00A200B492E
:10AD400008550CE0FDF744FA00680849095D405CCD
:10AD5000202804D10548005D303804490855601C9E
:10AD6000C4B2082CD2DBBDE8F08100005400002002
:10AD70000000B4435238A9422538640070B5054636
:10AD8000304800EB05142068804700283ED0207929
:10AD9000012802DA0120207152E02079022803DA2A
:10ADA0002079401C20714BE0A07A38B90120A072B4
:10ADB00005EB4501491CC8B200F08CFB2089002836
:10ADC0003EDDE088218988420DDAE088401C80B2AF
:10ADD000E0802189884233D105EB4501C91CC8B206
:10ADE00000F078FB2CE0E07A002829DD207B401C75
:10ADF000C0B22073E17A884222DB0020207305EB89
:10AE00004501491CC8B200F065FB19E02079012812
:10AE100002DD0120207110E0207918B12079401E58
:10AE200020710AE0A07A012807D10020A07205EB6A
:10AE30004501891CC8B200F04DFB0020E080207362
:10AE400070BD00008000002010B516480078401C3E
:10AE5000C0B214490870322810DB00200870124874
:10AE6000007B012804D11148006A0F49086103E002
:10AE70000E48006A0C49086100F084FD0A4A927A83
:10AE8000094B995C1A46907A00F0C0FC0648807A1B
:10AE9000401CC0B204498872082801DB0020887277
:10AEA00010BD00000100002054000020C000002060
:10AEB0000B48807A0A4AD27A904201D1002070472A
:10AEC0000748807A064A115C1046807A401CC0B25E
:10AED00090720A2801DB002090720846EFE700001C
:10AEE000B000002001460020244A914201D1C8143C
:10AEF00042E0234A914201D148143DE0214A914267
:10AF000002D14FF4002037E01F4A914202D14FF4A2
:10AF1000801031E01D4A914202D14FF400102BE025
:10AF2000B1F1804F01D1012026E0194A914201D1AF
:10AF3000022021E0174A914201D104201CE0164A68
:10AF4000914201D1082017E0144A914201D110200A
:10AF500012E0134A914201D120200DE0114A9142A2
:10AF600001D1402008E0104A914201D1802003E045
:10AF70000E4A914200D1881570470000002C014014
:10AF800000340140004C0140005001400054014099
:10AF90000004004000080040000C00400010004089
:10AFA0000014004000180040001C00400020004039
:10AFB0007047000010B54FF44070FEF771FD00F0CF
:10AFC000F9F800F07FF9FFF763F8FFF795F9012230
:10AFD00040210748FFF7B4F8FEF750FA00F0CCF82C
:10AFE00000F008F800F0D4F900F042F910BD0000BC
:10AFF0000038014008B501213020FEF789FD03200B
:10B000008DF8020010208DF803000120ADF800003B
:10B0100069463D48FEF73DFB0220ADF80000694659
:10B020003948FEF736FB0420ADF800006946364883
:10B03000FEF72FFB0820ADF8000069463248FEF706
:10B0400028FB1020ADF8000069462F48FEF721FBD1
:10B050002020ADF8000069462B48FEF71AFB40207F
:10B06000ADF8000069462848FEF713FB8020ADF8D4
:10B07000000069462448FEF70CFB4FF40070ADF861
:10B08000000069462148FEF704FB4FF48070ADF8DC
:10B09000000069461D48FEF7FCFA4FF48060ADF8E9
:10B0A000000069461948FEF7F4FA4020ADF80000A8
:10B0B00069461648FEF7EDFA4FF40060ADF800005F
:10B0C00069461148FEF7E5FA4FF48060ADF80000DC
:10B0D00069460D48FEF7DDFA4FF40070ADF8000048
:10B0E00069460948FEF7D5FA4FF48070ADF80000C4
:10B0F00069460548FEF7CDFA00F034F900F0FAF998
:10B1000000F040FC08BD00000014014000100140A8
:10B110007FB501210846FEF7EBFC1548006846089C
:10B120001448B6FBF0F085B24FF6FF74ADF8084056
:10B13000ADF804500020ADF80A00ADF8060001A9F2
:10B140004FF08040FEF700FF01218807FEF7D5FE93
:10B150001C208DF8000004208DF8010000208DF8DF
:10B16000020001208DF803006846FEF761FC7FBDF8
:10B170003C00002040420F0008B501210820FEF7E6
:10B18000C7FC03208DF8020014208DF80300402036
:10B19000ADF8000069460648FEF77BFA8020ADF85E
:10B1A000000069460248FEF774FA00F065FE08BD2B
:10B1B000000C014010B500F027F800F001F810BDB8
:10B1C00008B501214420FEF7A3FC03208DF80200FE
:10B1D00004208DF80300ADF8000069460848FEF72A
:10B1E00058FA0820ADF8000069460548FEF751FA04
:10B1F0000820ADF8000069460248FEF74AFA08BD8B
:10B2000000180140000801400021144A9172D172D7
:10B210001173002017E06421114A02EB0012118122
:10B2200000210F4A02EB001211710D4A02EB0012CD
:10B2300091720B4A02EB0012D172094A02EB001222
:10B240001173411CC8B20328E5DB0649044A1160AA
:10B25000054911610549116270470000B0000020E6
:10B2600080000020159800082D98000845980008D7
:10B2700008B501210420FEF74BFC4020ADF800008A
:10B2800010208DF8030003208DF8020069460B485A
:10B29000FEF7FFF9402009491431086000200849F1
:10B2A000087048608860087648760021044A116278
:10B2B00051629162D1621163516308BD000801407F
:10B2C000C000002070B5002416E0002004EB44010B
:10B2D000204A02EB8101486004EB440102EB81014A
:10B2E000886004EB440102EB8101487004EB4401E7
:10B2F00002F82100601CC4B2042CE6DB164800688A
:10B300004FF47A72B0FBF2F1B1F1807F00D31DE00F
:10B3100021F07F40401E4FF0E022506150170F2275
:10B32000002807DA13071E0E0C4B00F00F052D1F27
:10B330005E5503E013071D0E094B1D5400BF00208E
:10B340004FF0E02290610720106100BFFFF7E0FEA0
:10B3500070BD0000F80000203C00002018ED00E067
:10B3600000E400E0002000BF04E00B21074A115474
:10B37000411CC8B20828F8DB0021044A51729172BE
:10B38000D1721173116151619161704754000020B5
:10B3900008B501214FF4AC70FEF7BAFB03208DF81D
:10B3A000020010208DF80300C00240490860ADF88B
:10B3B000000069463D481038FEF76BF98020ADF873
:10B3C000000069463A48FEF764F94FF48060ADF832
:10B3D0000000694635481038FEF75BF94FF400600D
:10B3E000ADF80000694631481038FEF752F94FF4C5
:10B3F0000060ADF8000069462E48FEF74AF94FF4A8
:10B400008070ADF80000694628481038FEF741F911
:10B410008020ADF80000694624481038FEF739F95D
:10B420000220ADF8000069462348FEF732F90120FA
:10B43000ADF8000069462048FEF72BF94FF40050A4
:10B44000ADF80000694619481038FEF722F94FF4AC
:10B450008050ADF80000694614481038FEF719F91D
:10B460004FF48060ADF8000069461248FEF711F90C
:10B4700004208DF803000003ADF8000069460B4876
:10B480001038FEF706F9052000F030FB012000F02F
:10B4900003FB40F2DC5000F0A3FA4FF400600549D2
:10B4A00010310860012000F013FB08BD10180140A6
:10B4B00000100140000C01400020014010B50024A4
:10B4C00004E02046FFF75AFC601CC4B2032CF8DBF2
:10B4D00010BD00000649C97A054A50541146C97A80
:10B4E000491CC9B2D1720A2901DB0021D17270470F
:10B4F000B00000201CB504220021684600F06EFB5D
:10B500009DF8000055280ED19DF80100AA280AD107
:10B510009DF8020038B99DF80300FF2803D10020F0
:10B520000A49487211E09DF80000FF280DD19DF8EE
:10B53000010050B99DF80200AA2806D19DF8030029
:10B54000552802D10120014948721CBD5400002039
:10B5500010B5FFF7B3FFFDF7B5FF10BD10B5FFF74E
:10B5600073FC10BD2DE9FF5F04460D4691469A46D7
:10B570007448844202D07448844207D12046FFF7C1
:10B58000B1FC83460121FEF7C3FA06E02046FFF72F
:10B59000A9FC83460121FEF7ABFA002D41D1002121
:10B5A0002046FEF7AAFCAB466648844202D14FF023
:10B5B000190B28E0B4F1804F02D14FF01C0B22E0B0
:10B5C0006248844202D14FF01D0B1CE06048844267
:10B5D00002D14FF01E0B16E05E48844202D14FF0BC
:10B5E000320B10E05C48844202D14FF0360B0AE087
:10B5F0005A48844202D14FF0370B04E0524884424B
:10B6000001D14FF02C0B8DF800B08DF801908DF822
:10B6100002A000208DF803006846FEF709FABDE895
:10B62000FF9F484884420BD04748844208D04C488A
:10B63000844205D04B48844202D04B48844202D118
:10B640004A48066801E049480668642D0AD242F279
:10B650000F7842F21070B6FBF0F0B0FBF5F0401E30
:10B6600087B213E040F6B830854209D24FF0630844
:10B670006420B6FBF0F0B0FBF5F0401E87B205E0A9
:10B680004FF00008B6FBF5F0401E87B2ADF8087029
:10B69000ADF804800020ADF80A00ADF806008DF882
:10B6A0000C0001A92046FEF74FFC01212046FEF7C1
:10B6B00015FC012211462046FEF73CFC01212046E4
:10B6C000FEF71BFC4FF0000B1E48844202D14FF0E6
:10B6D000190B28E0B4F1804F02D14FF01C0B22E08F
:10B6E0001A48844202D14FF01D0B1CE018488442D6
:10B6F00002D14FF01E0B16E01648844202D14FF0E3
:10B70000320B10E01448844202D14FF0360B0AE0AD
:10B710001248844202D14FF0370B04E00A488442B9
:10B7200001D14FF02C0B8DF800B08DF801908DF801
:10B7300002A001208DF803006846FEF779F900BFEA
:10B740006DE70000002C014000340140000400407F
:10B7500000080040000C00400010004000140040B1
:10B76000004C014000500140005401403C000020CA
:10B77000416851B14168491E416031B901214170B0
:10B780000178012901D18168416070471CB51E48CC
:10B79000407A10B1012808D103E001201A4948720B
:10B7A00004E000201849487200E000BF00BF1648BE
:10B7B000407A012811D1FF208DF8000000208DF87B
:10B7C0000100AA208DF8020055208DF80300042204
:10B7D0000021684600F041FA13E00B48407A80B936
:10B7E00055208DF80000AA208DF8010000208DF86A
:10B7F0000200FF208DF8030004220021684600F0BB
:10B800002CFA00F0BFF81CBD54000020202900D104
:10B810000B210C2900DB704700BF4FF40072554B21
:10B820005A6152105A6192005A6140225A61520183
:10B83000514B1A6052101A6052101A6052101A605E
:10B8400000BF00BF01221A6002221A6004221A609F
:10B8500008221A6010221A6020221A6040221A6000
:10B8600080221A6000BFC1EBC102444B9A5C1AB13E
:10B870000122414B1B1F1A60C1EBC1023F4B1A440E
:10B8800052781AB102223C4B1B1F1A60C1EBC10255
:10B890003A4B1A4492781AB10422374B1B1F1A6094
:10B8A000C1EBC102354B1A44D2781AB10822324B8F
:10B8B0001B1F1A60C1EBC102304B1A4412791AB136
:10B8C00010222D4B1B1F1A60C1EBC1022B4B1A44D7
:10B8D00052791AB12022284B1B1F1A60C1EBC102FA
:10B8E000264B1A4492791AB14022234B1B1F1A602F
:10B8F000052807D1224A527A012A03D180221E4B01
:10B900001B1F1A60082830D2DFE800F004090E136C
:10B91000171D23294FF40072164B1A6126E04FF4CD
:10B920008072144B1A6121E04FF48062114B1A614E
:10B930001CE040220F4B1A6118E04FF400620E4BDE
:10B940001B1F1A6012E04FF480620B4B1B1F1A6022
:10B950000CE04FF40072084B1B1F1A6006E04FF416
:10B960008072054B1B1F1A6000E000BF00BF00BFC4
:10B9700051E700000010014014140140ACC700085A
:10B980005400002010B500241448C07A18B11348A0
:10B99000C07A02281BD11148407A28B90A2208210E
:10B9A0000E48FCF734FC18E00C48407A012814D10A
:10B9B000002404E00B2009490855601CC4B2052C82
:10B9C000F8DB0A20054948718871C87105E0034811
:10B9D000C07A012801D1FFF755F910BD54000020AD
:10B9E0002DE9F04786B004462046FCF7A7FF8146C4
:10B9F00001210420FEF78CF801214807FEF778F8B2
:10BA00001020ADF8140000208DF8170003208DF8E9
:10BA1000160005A91D48FDF73CFE10211B48FDF747
:10BA2000C3FE00200190029003900220049001A91F
:10BA30000020FDF7C9FD01210020FDF7B1FD002127
:10BA40000846FDF7DBFD12494846FCF74FFE8146EC
:10BA50004FF08B414846FCF717FE8246FCF7C1FFCA
:10BA600007464FF066320B4BFCF7F0FE0546FCF73D
:10BA7000CBFF81464846FCF77FFF85B22946002070
:10BA8000FDF7BCFD06B0BDE8F087000000080140EE
:10BA900000007A4466660A4010B1012811D107E01F
:10BAA0004FF48061084A11600021084A117309E0CF
:10BAB0004FF48061044A121F11600121034A11737F
:10BAC00000E000BF00BF7047141801405400002080
:10BAD00020B94FF40061044A116004E04FF40061A2
:10BAE000014A121F116070471418014006286FD2D6
:10BAF000DFE800F00315283B4D5D3749096821F068
:10BB00007041354A11601146096841F04051116099
:10BB10009115314A143211608021116059E02E498B
:10BB2000096821F070412C4A11601146096841F002
:10BB3000405111609115284A143211608021121F62
:10BB4000116046E02449096821F07041224A1160E1
:10BB50001146096841F04051116091151E4A10329A
:10BB600011608021121D116033E01B49096821F02A
:10BB70007041194A11601146096841F04051116045
:10BB80009115154A103211608021116021E012498F
:10BB9000096821F07041104A11601146096841F0AE
:10BBA0008041116091150C4A1432116011E00A496C
:10BBB000096821F07041084A11601146096841F096
:10BBC000804111609115044A1032116001E0FFE7D5
:10BBD00000BF00BF70470000001801402DE9F04190
:10BBE00007460D46164600F02FF9A02000F002F996
:10BBF00000F054F900B12CE0281200F0FBF800F03E
:10BC00004DF900B125E0E8B200F0F4F800F046F993
:10BC100000B11EE000F018F9A12000F0EBF800F0F0
:10BC20003DF900B115E000240CE000F0C1F83855F2
:10BC3000701EA04202D000F087F801E000F0A4F8E6
:10BC4000601C84B2B442F0DB00F016F90120BDE8BC
:10BC5000F08100F011F90020F9E72DE9F0470746DF
:10BC6000884691464546002433E014B105F03F0074
:10BC700020BB00F001F900260AE000F0E5F8A02062
:10BC800000F0B8F800F00AF900B904E0701C86B2C0
:10BC9000B6F57A7FF1DB00BFB6F57A7F00D11FE001
:10BCA000281200F0A7F800F0F9F800B118E0E8B2A7
:10BCB00000F0A0F800F0F2F800B111E0385D00F0FB
:10BCC00099F800F0EBF800B10AE0681C85B2601C3E
:10BCD00084B24C45C9DB00F0CFF80120BDE8F08705
:10BCE00000F0CAF80020F9E770B504460D46E1B24D
:10BCF0000548FEF7FCFA00BF80210348FEF729FA49
:10BD00000028F9D0204670BD0038014070B50024ED
:10BD10000A210120FDF764FD05462C4640F6B830A7
:10BD2000844201DD02240CE0B4F5966F01DC0124AD
:10BD300007E0B4F5966F04DD40F6B830844200DCCD
:10BD40000024204670BD000010B58020094908601D
:10BD500000F012F840200749091F086000F00CF8B5
:10BD600040200449086000F007F880200149091FBD
:10BD7000086010BD140C0140002001E0411CC8B255
:10BD80001E28FBDB7047000010B5802007490860C3
:10BD9000FFF7F2FF402005490860FFF7EDFF402064
:10BDA0000249091D0860FFF7E7FF10BD100C0140B4
:10BDB00070B50024002516E06006040E40200C49F2
:10BDC0000860FFF7D9FF0A480838006800F08000D3
:10BDD00008B1601CC4B240200549091D0860FFF786
:10BDE000CBFF681CC5B2082DE6DB204670BD000005
:10BDF000100C014070B50446002520E004F08000DE
:10BE000018B180200F49086003E080200D49091D0A
:10BE10000860FFF7B1FF40200A490860FFF7ACFF58
:10BE200040200849091D0860072D02D18020091F04
:10BE300008606006040EFFF79FFF681CC5B2082D5E
:10BE4000DCDB70BD100C014010B580200949086092
:10BE500040200860FFF790FF80200649091D086018
:10BE6000FFF78AFF40200349091D0860FFF784FFA0
:10BE700010BD0000100C014010B58020064908607C
:10BE80004020091F0860FFF777FF80200249091F43
:10BE90000860FFF771FF10BD140C014010B5802041
:10BEA0000C490860FFF768FF40200A490860FFF767
:10BEB00063FF08480838006800F0800008B10124DA
:10BEC00000E0002440200349091D0860FFF754FFEB
:10BED000204610BD100C014008B540F2DC58002788
:10BEE000002500264A484B49086001210420FDF73F
:10BEF0000FFE4FF48070ADF8000018208DF803009D
:10BF000003208DF8020069464348FDF7C2FB434811
:10BF1000406840F0E060414948600846406800F0F1
:10BF20000C05082D04D108464068C0F38346B61CB2
:10BF3000FFF740F81DB93AA0FEF712FA0DE0042D04
:10BF400003D13CA0FEF70CFA07E0082D05D1F30061
:10BF5000324631463BA0FEF703FA4448016844A04C
:10BF6000FEF7FEF92D484068C0F302222B484168D5
:10BF700046A0FEF7F5F94E48828D018D4DA0FEF7E3
:10BF8000EFF9FDF735FA01231A4614214046FDF773
:10BF9000EDFA01204E49C872FDF70EFD36E0FFF7BD
:10BFA00007F800F041FA4B48007801281AD1002028
:10BFB00048490870FFF7AAFE0746012F08D100275D
:10BFC00040F6B83200231946501000F085F809E019
:10BFD000022F07D1002740F6B8320023012150106C
:10BFE00000F07AF8FEF764FF0446002C0EDD012C09
:10BFF00002D0042C08D102E0FDF7FCFC05E0FDF7BF
:10C0000057FAFFF7C3FB00E000BF00BFC7E700001F
:10C010000080000808ED00E0000801400010024028
:10C02000535953434C4B203D2048534920384D48E9
:10C030007A0D0A00535953434C4B203D2048534539
:10C040000D0A0000504C4C204D554C203D202575CC
:10C050002C20504C4C203D20384D487A202A202559
:10C0600075203D2025754D487A0D0A003C000020C2
:10C0700053797374656D436F7265436C6F636B20A6
:10C08000766172203D20256C750D0A005243432DC8
:10C090003E43464752203D2030782530386C582C9E
:10C0A0002050505245313D256C750D0A00000000AE
:10C0B0000010004054494D3620505343203D202568
:10C0C000752C20415252203D2025750D0A0000009C
:10C0D00054000020000000202DE9F04107460C46E6
:10C0E00015461E462B48C07A012850D1012C17D185
:10C0F00000BF2949D1E90A01643041F100016FF024
:10C100000042514071EA000020D02348D0E90A30B3
:10C1100064229A1840F100001F49C1E90A2015E085
:10C12000A4B900241C49D1E90A01643861F1000175
:10C130004FF000425140084308D01748D0E90A2088
:10C14000643A60F100001449C1E90A201248D0E9BC
:10C150000810114AD2E90A32C91A904107DA00BF21
:10C160006422002140F2DC50FDF7FCFB0FE00A489E
:10C17000D0E90A200849D1E90831D21A884106DA03
:10C1800000BF6422012140F2DC50FDF7EBFBBDE86B
:10C19000F081000054000020C000002010B519A05C
:10C1A000FEF7DEF818A0FEF7DBF820A0FEF7D8F8BF
:10C1B00029A0FEF7D5F82FA131A0FEF7D1F836A1BE
:10C1C00038A0FEF7CDF83DA0FEF7CAF845A0FEF76F
:10C1D000C7F84DA0FEF7C4F851A0FEF7C1F858A06B
:10C1E000FEF7BEF860A0FEF7BBF86AA0FEF7B8F84D
:10C1F0007048FEF7B5F87048FEF7B2F86FA0FEF78A
:10C20000AFF810BD0D0A00002D2D2D2D2D2D2D2D3B
:10C210002D2D2D2D2D2D2D2D2D2D2D2D2D2D2D2D4E
:10C220002D2D2D2D2D3E0D0A000000002D3E20E865
:10C23000AEBEE5A487E5908DE7A7B0EFBC9AE69780
:10C24000A0E99990E6978BE8BDACE68EA7E588B6A5
:10C25000E599A80D0A0000002D3E20736F667477E3
:10C2600061726520766572736F6E3A2056312E309A
:10C270000D0A000031363A32373A313600000000FC
:10C280002D3E20636F6D70696C652074696D653A31
:10C290002025730D0A0000004170722031362032D3
:10C2A000303236002D3E20636F6D70696C652064FE
:10C2B0006174653A2025730D0A0000002D3E205B55
:10C2C000E5A49AE59CBAE4BD8EE6B8A9E7A791E695
:10C2D0008A80E69C89E99990E585ACE58FB85D0D8B
:10C2E0000A0000002D2D2D2D2D2D2D2D2D2D2D2D28
:10C2F0002D2D2D2D2D2D2D2D2D2D2D2D2D2D2D2D6E
:10C300002D2D0D0A000000002D3EE58FAFE794A80B
:10C31000E591BDE4BBA4EFBC9A5C720A000000008A
:10C32000312E205B735D20202F2F20E5819CE6AD10
:10C33000A2E794B5E69CBAE8BDACE58AA80D0A0070
:10C34000322E205B3F5D20202F2F20E8AFBBE58FF2
:10C3500096E5BD93E5898DE4BD8DE7BDAEE8A79276
:10C36000E5BAA60D0A000000332E205B7A5D20207E
:10C370002F2F20E8AEBEE7BDAEE5BD93E5898DE485
:10C38000BD8DE7BDAEE4B8BAE99BB6E782B95C7291
:10C390000A000000342E205B4D465D202F2F20E642
:10C3A0008993E58DB0E7B3BBE7BB9FE4BFA1E6810E
:10C3B000AF0D0A0088C80008D8C800083C2D2D2DF4
:10C3C0002D2D2D2D2D2D2D2D2D2D2D2D2D2D2D2D9D
:10C3D0002D2D2D2D2D2D2D2D2D2D0D0A0000000084
:10C3E00070B50B490869FCF7A0FA06460949FCF745
:10C3F0004BF905460849FCF779F904462046FCF755
:10C40000F0FA05462A460B4604A0FDF7A9FF70BDC9
:10C41000540000200000B443003404465B772C2510
:10C420002E32665D0D0A00002DE9F04387B000242E
:10C430000020069000250590A148007800281BD018
:10C4400000209F4908709F48FBF7F3FEC4B2032CFD
:10C4500013D19C4840783F2804D0732805D07A280F
:10C4600009D105E0FFF7BCFF06E0FDF7A5FA03E000
:10C47000FDF7C0FA00E000BF1EE1042C0AD191488C
:10C4800040784D28F8D18F4880784628F4D1FFF7BE
:10C4900085FE11E18B484078722878D105AB06AA59
:10C4A00089A18848FBF7CCFE022876D189490698F5
:10C4B000FCF7C6FA02D28748069006E0864906983D
:10C4C000FCF7C8FA01D28448069084490598FCF725
:10C4D0000DF906468249FCF7D7F8054681490698CA
:10C4E000FCF7D2F806902846FCF75AFA7E4AC2E9D1
:10C4F0000A012846FCF727FA06460598FCF771FA68
:10C50000074688460698FCF737FA81467648C16A9E
:10C51000806A3A4643460096CDE90201494673A037
:10C52000FDF71EFF7E48828D018D7EA0FDF718FF6E
:10C530006D48D0E908306C4AD2E90A12591A904184
:10C5400008DA0698FCF718FA06467B220021FDF768
:10C5500009FA18E06448D0E90A10634BD3E90823CC
:10C56000891A984108DA0698FCF706FA06467B22F3
:10C570000121FDF7F7F906E003230522114640F2F9
:10C58000DC50FCF7F3FF6648828D018D01E08CE002
:10C5900003E06DA0FDF7E4FE8EE005AB06AA73A1F3
:10C5A0004848FBF74DFE022877D14A492846FCF758
:10C5B00047FA01D2474D05E047492846FCF74AFAB9
:10C5C00000D2454D45490598FCF790F80646444988
:10C5D000FCF75AF8054643490698FCF755F80690CB
:10C5E0002846FCF7DDF9404AD2E90A32C018514129
:10C5F0003D4AC2E90A012846FCF7A5F90646059816
:10C60000FCF7EFF9074688460698FCF7B5F981462E
:10C610003548C16A806A3A4643460096CDE9020130
:10C62000494655A0FDF79CFE3D48828D018D3DA0F9
:10C63000FDF796FE2C48D0E908102B4AD2E90A32C1
:10C64000C91A904108DA0698FCF796F906467B224B
:10C650000021FDF787F918E02348D0E90A10224AA3
:10C66000D2E90832C91A904108DA0698FCF784F931
:10C6700006467B220121FDF775F906E0032305221A
:10C68000114640F2DC50FCF771FF2548828D018D88
:10C690002DA0FDF765FE0FE0FFE7032305221146FD
:10C6A00040F2DC50FCF762FF06E00323052211464E
:10C6B00040F2DC50FCF75AFF07B0BDE8F083000001
:10C6C00025000020680100205B723A25663A256645
:10C6D0005D0000000AD7233C0000C8430000B443BB
:10C6E00000340446B005BC41C00000205B725D20F0
:10C6F000667265713D256C752C20616E676C653DB9
:10C7000025662C2070756C73653D256C642C207338
:10C71000765F70756C73653D256C6C640D0A000066
:10C720000010004054494D36206265666F726520E6
:10C7300073746172743A205053433D25752C204127
:10C7400052523D25750D0A0054494D3620616674DC
:10C7500065722073746172743A205053433D25759D
:10C760002C204152523D25750D0A00005B72723A31
:10C7700025663A25665D00005B72725D2066726513
:10C78000713D256C752C20616E676C653D25662CAE
:10C790002070756C73653D256C642C2073765F701A
:10C7A000756C73653D256C6C640D0A000101010117
:10C7B0000101000001010000000001010001010071
:10C7C000010101010100000100010100000101015E
:10C7D000000101000101010001010101010101014C
:10C7E000000000000101010101010101010101003E
:10C7F0000101000000000000010000000000000036
:10C800000040404040404040404041414141414063
:10C810004040404040404040404040404040404018
:10C8200040050202020202020202020202020202A7
:10C8300002202020202020202020200202020202AC
:10C840000202909090909090101010101010101004
:10C850001010101010101010101010100202020210
:10C860000202888888888888080808080808080854
:10C870000808080808080808080808080202020250
:10C880004000000001C80008352E205B723A3130AC
:10C890003A3336305D202F2F20E8BDACE58AA8E57D
:10C8A00091BDE4BBA4EFBC8C3130E4B8BAE8BDACB8
:10C8B000E58AA8E8A792E9809FE5BAA6EFBC8C3389
:10C8C0003630E4B8BAE79BAEE6A087E8A792E5BAAF
:10C8D000A65C720A00000000362E205B72723A31AC
:10C8E000303A32305D202F2F20E8BDACE58AA8E534
:10C8F00091BDE4BBA4EFBC8C3130E4B8BAE8BDAC68
:10C90000E58AA8E8A792E9809FE5BAA6EFBC8C3239
:10C9100030E4B8BAE79BB8E5AFB9E8BDACE58AA8A2
:10C92000E8A792E5BAA65C720A0000004CC90008AC
:10C930000000002054000000B4A30008A0C90008B3
:10C940005400002054810000C4A30008000000002F
:10C9500000000000000000000000000000000000D7
:10C9600000000000000000000000000000000000C7
:10C970000000000000000102030401020304060796
:10C98000080902040608000000A24A040000000092
:10C99000000000000102030406070809000000006F
:04000005080081313D
:00000001FF
